:020000040000FA
:02000000B7291E
:02000800382E90
:10001000831203134808E1000130E2004908031984
:100020001528E20D6210FF3E0F286208E300E20986
:1000300080304807840062088005841362088005C8
:100040000800C920E830F4000330F500F601F7019C
:10005000D2204A08F4004B08F500F601F701FE2013
:10006000F30CF20CF10CF00CF313F30CF20CF10C9A
:10007000F00CF313F30CF20CF10CF00CF31370080A
:10008000E4007108E500C9204C08F4004D08F500B3
:10009000F601F701D2206408F4006508F500F601C6
:1000A000F7010330003E03195C28F40DF50DF60D41
:1000B000F70D7410FF3E5328FE207008E800710809
:1000C000E9007208EA007308EB000A30F40000301F
:1000D000F5006408F0006508F10087217008E4006D
:1000E0007108E50000307102031D782803307002AA
:1000F00003187B280800610884006B08003C031D7E
:100100008B286A08003C031D8B286908003C031DEE
:100110008B286808003C0318C6286308800465081B
:100120000319A228E601E70166086702031D9A2861
:10013000650866020318A228EC01A421E60A031947
:10014000E70A94286408EC00A42162088005650889
:100150000319BA28E601E70166086702031DB22801
:10016000650866020318BA28EC01A421E60A0319FF
:10017000E70AAC286408EC00A4210130E802031C63
:10018000E902031CEA02031CEB027D2862088005D9
:100190000800831203130030F0003230F100F20146
:1001A000F3010800831203132230FC00F801F90167
:1001B000FA01FB01FC030319EE280310FB0CFA0CF7
:1001C000F90CF80CF30CF20CF10CF00C031CDA280F
:1001D000FC030319ED28EF20DE28EF200800740847
:1001E000F80775080318750FF90776080318760FD6
:1001F000FA0777080318770FFB0708008312031329
:10020000FB01FA01F901F801E001730DF80D740822
:100210006321F30D0730FC00730D5D217408731C1E
:100220001329632114297521F30DFC0B0C29720D80
:100230005D217408731C1E2963211F297521F20D8D
:100240000730FC00720D5D217408721C292963219E
:100250002A297521F20DFC0B2229710D5D217408EC
:10026000721C3429632135297521F10D0730FC00FA
:10027000710D5D217408711C3F296321402975218E
:10028000F10DFC0B3829700D5D217408711C4A2991
:1002900063214B297521F00D0730FC00700D5D21A5
:1002A0007408701C5529632156297521F00DFC0B2B
:1002B0004E2970185C29EF200800F80DF90DFA0D91
:1002C000FB0DE00D0800F8027508031C750FF9021C
:1002D0007608031C760FFA027708031C770FFB02DF
:1002E0000301031C0130E0020800F8077508031839
:1002F000750FF90776080318760FFA0777080318C1
:10030000770FFB07030103180130E0070800831291
:100310000313F801F9011030FC00710DF80DF90D0F
:100320007408F8027508031C750FF90203189F2959
:100330007408F80775080318750FF9070310F00D16
:10034000F10DFC0B8D29080083120313EC03EC0361
:100350006C08003C0318B129EC0300000000000009
:10036000A82900000000000000000000080083121F
:1003700085018601870183160C10D13081000B3076
:100380008500003086008617F030870005309F001A
:10039000831220308B0080309F000630C800073069
:1003A000C9000820CE01203084000530C5000317A5
:1003B00026308D00031783160C1483120C088D0A47
:1003C00003138000840AC50BDA29A501B701B8011F
:1003D000A901AA01AB01BC018B177F3086002F2237
:1003E00050226D22BC30B1000230B2004030B30068
:1003F000DD30A7002910A5013130BE00CB24033029
:100400002502031CFC297F308600A501013025024E
:10041000031C062AB101B201B301FC30A700291068
:10042000A8013130BE000630AA001A30AB00CB2440
:100430000130A806031D112A993031020319252A1B
:100440001130B107B207B307112A7F308600A5012A
:1004500001302502031C282AA501B901032B103005
:10046000CA000330CB006430CC000030CD008316CE
:100470008613831221208316861783121E302726A7
:100480001730CA000430CB006430CC000030CD00FF
:100490008316861383122120831686178312080081
:1004A000003085000030C1008822B0220930C10030
:1004B0009C22D9220A30C1008822C1220430C10006
:1004C0009C22EA22203085000530C1008822B0221B
:1004D0000E30C1009C22D92208000330C600003033
:1004E00085000030C1008822B0220A30C100C1223C
:1004F0000530C100B0220E30C1009C22D922043048
:10050000C100EA220930C100D922C60B6F2A0800B7
:100510008700FE30C2000730C5007F30860005121C
:10052000451C051642087F3986001430272603141F
:10053000C20DC50B8D2A08008700BF30C2000730EE
:10054000C5007F3086000516451C051242087F391C
:100550008600143027260314C20CC50BA12A0800FC
:100560000A30C5007F3086000512451C051641087B
:1005700087003F30860014302726C10AC50BB22AF7
:1005800008000A30C50005304502031DCA2A203084
:100590008500C1017F3086000512451C0516410803
:1005A00087003F30860014302726C10AC50BC32AB6
:1005B00008000A30C5007F3086000512451C05166C
:1005C000410887007E30860014302726C103C50B02
:1005D000DB2A08000A30C50005304502031DF42A55
:1005E000003085000E30C1007F3086000512451CAA
:1005F0000516410887007E30860014302726C10387
:10060000C50BEC2A0800A919AD23E32300303702FB
:1006100003190E2B04303702031D1B2B1324FE304D
:10062000A7003A1C572B3E0884000008F039031934
:10063000A713CB23572B01303702031D252B203066
:10064000BE00FD30A700D723572B02303702031D11
:10065000362BF9233130BE003D30A7001030320276
:10066000031CA7120A30B304D723572BFB302507EE
:10067000031C0E2BF6302507031C1F2BE03025072B
:10068000031C0E2BDB302507031C292BCB30250741
:10069000031C0E2BC6302507031C1F2BB03025076B
:1006A000031C0E2BAB302507031C292B0E2BCB2450
:1006B0004E1C6A2B7030CA000330CB006430CC0073
:1006C0000030CD00831686138312212083168617EF
:1006D00083127B2BCE1C7B2BE030CA000630CB0074
:1006E000E830CC000330CD0083168613831221201E
:1006F000831686178312CE01BC1F852BB70A0530DF
:1007000037020319B701B8179C2B3C1F892B3C24D7
:100710009C2B3C1E9C2B06302402031C962B553030
:100720002402031C9C2B8B137B26972B8B13A40179
:10073000A501AA01AB018B17BC01A91C032B8125C4
:10074000A910A91501302202031D032BC325013076
:100750002102031D032BD525032BA9112030840072
:100760000530C500031726308D0003130008840AE6
:1007700003178C0083168C130C1555308D00AA308E
:100780008D008C148C18C22B0C1183128D0A03134C
:10079000C50BB62B08003A18D32B281412302302AD
:1007A00003182810D62B2814BA18281008003A1855
:1007B000DF2B28101230230203182814E22B2810F4
:1007C000BA182814080083169F13831281309F00E3
:1007D0001E261F151F19EA2B76301E020318F22B56
:1007E0002915F72B8A301E02031CF72B29111F1025
:1007F000080083169F17831289309F001E261F153D
:100800001F19002C1E08AC0083161E088312AD00B1
:100810001F10A5263308B200B20E3408B204350802
:10082000B300B30E0800BA01831685178312233074
:10083000861B3A2C2308B1002408B2002508B30017
:100840003A143108031D272C1230B100392C123014
:100850003102031C392CBA140319392CB1000E30A3
:100860003102031C392C103031020318392C0630A8
:10087000B1023130BE0008008B130530B700B81349
:100880002008AE002108AF002208B0002030BE00D2
:10089000C130A700D723CB24BC1B992C3C1B582C60
:1008A000BC1E542CD525482C3C1E482C0226482C16
:1008B0003130A700D723CB24BC1B482C3C1B6A2C0F
:1008C000BC1E642CC325582C3C1E582CF625582CD5
:1008D0002030BE000D30A700D723CB24BC1B582CE2
:1008E0003C1B7A2CBC1E762C81256A2C3C1E6A2C63
:1008F000E6256A2C1324C230A700CB23CB24BC1BD3
:10090000682C3C1B992CBC1E8D2C23308400852622
:10091000243023020318A3017A2C3C1E7A2C2330A6
:1009200084001326F9302302031D7A2C2330A30000
:100930007A2C13243230A700CB23CB24BC1B7A2C77
:100940003C1BB82CBC1EAC2C2430840085266030A7
:1009500024020318A401992C3C1E992C24308400F5
:100960001326F9302402031D992C5930A400992C28
:1009700020082E02031DC42C21082F02031DC42CA5
:10098000220830020319C52CA915B701AA01AB0131
:10099000A5018B17080005303702031DD02CBC01C0
:1009A00000302818103085003E088400B81BDA2C6F
:1009B000A71FDF2CC101B81BC117000E4325271F3D
:1009C000E52C0530C10000084325840AA71EEC2C45
:1009D0000A30C100000E4325203028183030850031
:1009E000271EF52CC10100084325840AA71DFC2CF5
:1009F0000530C100000E4325271D022D0A30C1001D
:100A0000000843257F30860004308500A71C1C2D7C
:100A10000F303A1C272D05303702031D142D0B30E3
:100A2000BA1C272D0730272D0F303B1C272D0730F0
:100A3000BA1C272D0B30272D0030271C272D053001
:100A400037020319262D0130271F272D0530FF3AC5
:100A50007F39860020267F308600BD080319322D9D
:100A6000BD033B2D0708F039F03ABC0003193B2DBC
:100A70009630BD002914053037020319422D291C78
:100A8000CB2C291008000F39C400C500C11B542D00
:100A90000630C3000310C40DC40D4508C407D73089
:100AA000C4070318C30A602D3708C500C50AFE3005
:100AB000C700C713C5030319602D0314C70D592DB3
:100AC0000530C5007F308600291D672D222641088C
:100AD0000F398700C11B712D7D257F39C700053077
:100AE0008A00470886002026C10AC40A0319C30ADF
:100AF000C50B622D7F308600080043088A00440839
:100B00008200A20A2208A6000F30A6050A3026029B
:100B1000031D8C2D0630A2079625A600220826026A
:100B2000031C932D08000130A200080002302102AE
:100B3000031DAF2D200E0F39A6000310A60DA60D24
:100B4000A607A60D20080F3926070339031DAB2D74
:100B50002008031DAD2D2830C22D2930C22D0430B0
:100B600021020319C12D063021020319C12D0930BC
:100B700021020319C12D113021020319C12D313079
:100B8000C22D30300800A10A2108A6000F30A605AA
:100B90000A302602031DCE2D0630A1071330210294
:100BA000031CD42D0130A1000800A00A2008A600D3
:100BB0000F30A6050A302602031DE02D0630A007DF
:100BC000A0302002031CE52DA0010800A203031998
:100BD000F32D2208A6000F30A6052602031D0800EB
:100BE0000630A20208009625A2000800A103031DFA
:100BF000FB2D1230002E0F302102031D080009309A
:100C0000A1000800A003FF302002031D092E66305A
:100C1000112E2008A6000F30A6052602031D08008D
:100C20000630A002080080030008B6000F30B605A9
:100C30003602031D08000630800208001630232EFD
:100C40003430232E6930BF00BF0B242E0800BF00B4
:100C50000030C000000000000000000000000000A4
:100C6000000000000000C00B2A2EBF0B282E080039
:100C7000FD00030E8301FE000A08FF008A0104083C
:100C8000ED000B19442E622E0B11AB0F482EAA0A51
:100C900035302B02031D622E0C302A02031C622EFB
:100CA0000130BB06AA01AB016B26291439080319D0
:100CB0005D2EB90B612EB813612EB81F612E023064
:100CC000B90091266D0884007F088A007E0E83009B
:100CD000FD0E7D0E0900253084008526603025023A
:100CE000031C0800A50124308400852660302402FE
:100CF000031C0800A401233084008526243023022D
:100D0000031C0800A914A3010800800A0008B6000B
:100D10000F30B6050A303602031D08000630800782
:100D2000080004303702031DA42E59302402031D8D
:100D30009F2E57302502031C9F2E4E14A42E2508EB
:100D40002404031DA42ECE1408002C0E0F39F03EEF
:100D5000B200B207E23EB300323EB5002C080F39B4
:100D6000B307B307B507E93EB400B407B4072D0EC7
:100D70000F39B407B507B40DB50DB509B50D2D087C
:100D80000F39B507B20D0730B1000A30B507B4030B
:100D9000031CC62EB407B303031CCA2EB307B20349
:100DA000031CCE2EB207B103031CD22E0800C1349F
:100DB000BE34BE34BE34C134FF34DE348034FE343D
:100DC000FF34DE34BC34BA34B634CE34BD34BE3431
:100DD000AE349634B934F334EB34DB348034FB3442
:100DE0008D34AE34AE34AE34B134E134D634B634AE
:100DF000B634F934BF34B834B734AF349F34C9345F
:100E0000B634B634B634C934CF34B634B634B53467
:100E1000C33491348E34EE34EE34FD348334FD34F7
:100E2000FE34FD348334F134EA34F334E034F734FF
:02400E00723FFF
:1042000043006F0070007900720069006700680069
:1042100074002000280043002900200032003000F4
:10422000300037002D00320030003100390020000E
:104230006200790020004D002E00590061006D00E1
:1042400061006D006F0074006F00FF001400090032
:0642500001000000000067
:00000001FF
